:0200000480007A
:10000000971F0000938F0F00171100001301810349
:1000100083D10F0003D22F0023203100232241007F
:10002000171C0000130C5CFE971200009382020262
:10003000835CFCFF035D1C0023A0920123A2A201AC
:1000400097130000938373FC1714000013048400BB
:1000500003DF130083DF33002320E4012322F401B4
:10006000171500001305C57A97150000938505FF45
:10007000035605808356258023A0C50023A2D50002
:10008000970600009386367917170000130787FD3F
:1000900083D7D67F03D8F67F2320F70023220701DA
:1000A00017180000130888F797180000938808FCB9
:1000B0000359C8FF8359E8FF035A0800835A2800F0
:1000C000035B4800835B680023A0280123A238015A
:1000D00023A4480123A6580123A8680123AA780174
:1000E000971A0000938A0AF4171B0000130B8BF970
:1000F00003D00A0023200B00971A0000938ACAF24B
:10010000171B0000130B4BF883AB0A0003DC0B003A
:10011000930C0C0023209B01971C0000938C4CF146
:10012000171D0000130D8DF683DC0C0023209D01AC
:10013000971D0000938D1DF0171E0000130E4EF545
:1001400083DDFDFF2320BE0117150000130585EF99
:1001500097150000938505F4370610F01306C6F2D4
:100160006306B5028326C5002320D60083268500BA
:100170002320D600832645002320D60083260500B1
:100180002320D600130505016FF09FFD370510F001
:10019000130505F223200500000000000000000008
:0401A000000000005B
:1010000022F2F111F44433F366F6F555F88877F7D8
:10101000AA0A09990CCCBB0BEE0E0DDDF000FF0FF8
:101020007856341228100080F0DEBC9A10325476C4
:1010300098BADCFE00000000000000000000000084
:10104000FFFFFFFFFFFFFFFFFFFFFFFFFFFFFFFFB0
:10105000FFFFFFFFFFFFFFFFFFFFFFFFFFFFFFFFA0
:10106000FFFFFFFFFFFFFFFFFFFFFFFFFFFFFFFF90
:10107000FFFFFFFFFFFFFFFFFFFFFFFFFFFFFFFF80
:10108000FFFFFFFFFFFFFFFFFFFFFFFFFFFFFFFF70
:040000058000000077
:00000001FF
